S025000062696E2F64656D6F70726F675F6F6C696D65785F73746D3332703430352E737265632C
S31508008000000002205D820008AB820008AD820008ED
S31508008010AF820008B1820008B382000800000000A1
S31508008020000000000000000000000000B582000803
S31508008030B782000800000000B98200088D87000892
S31508008040BF820008C1820008C3820008C5820008F2
S31508008050C7820008C9820008CB820008CD820008C2
S31508008060CF820008D1820008D3820008D582000892
S31508008070D7820008D9820008DB820008DD82000862
S31508008080DF820008E1820008E3820008E582000832
S31508008090E7820008E9820008EB820008ED82000802
S315080080A0EF820008F1820008F3820008F5820008D2
S315080080B0F7820008F9820008FB820008FD820008A2
S315080080C0FF8200080183000803830008058300086F
S315080080D007830008098300080B8300080D8300083E
S315080080E00F8300081183000813830008158300080E
S315080080F017830008198300081B8300081D830008DE
S315080081001F830008218300082383000825830008AD
S3150800811027830008298300082B8300082D8300087D
S315080081202F8300083183000833830008358300084D
S3150800813037830008398300083B8300083D8300081D
S315080081403F830008418300084383000845830008ED
S3150800815047830008498300084B8300084D830008BD
S315080081604F8300085183000853830008558300088D
S3150800817057830008598300085B8300085D8300085D
S315080081805F83000861830008EE11AA5510B5054CF7
S31508008190237833B9044B13B10448AFF300800123A5
S315080081A0237010BD7C00002000000000608F0008CE
S315080081B0084B10B51BB108490848AFF300800848BA
S315080081C0036803B910BD074B002BFBD0BDE8104070
S315080081D0184700BF0000000080000020608F0008DC
S315080081E07C00002000000000154B002B08BF134B35
S315080081F09D46A3F5803A00218B460F461348144A3C
S31508008200121A00F085FE0F4B002B00D098470E4B34
S31508008210002B00D098470020002104000D000D48CF
S31508008220002802D00C48AFF3008000F04BFE200077
S31508008230290000F02DFA00F031FE00BF000008000A
S315080082400000022000000000000000007C00002062
S31508008250F0000020000000000000000007498D46DD
S315080082600749084A084B9A42BEBF51F8040B42F820
S31508008270040BF8E705488047054800470000022038
S315080082806C8F0008000000207C000020518E00083A
S31508008290E98100083349344A002301E041F8043BE8
S315080082A09142FBD300F0F4F9FEE7FEE7FEE7FEE7AE
S315080082B0FEE7FEE7FEE7FEE7FEE7FEE7FEE7FEE788
S315080082C0FEE7FEE7FEE7FEE7FEE7FEE7FEE7FEE778
S315080082D0FEE7FEE7FEE7FEE7FEE7FEE7FEE7FEE768
S315080082E0FEE7FEE7FEE7FEE7FEE7FEE7FEE7FEE758
S315080082F0FEE7FEE7FEE7FEE7FEE7FEE7FEE7FEE748
S31508008300FEE7FEE7FEE7FEE7FEE7FEE7FEE7FEE737
S31508008310FEE7FEE7FEE7FEE7FEE7FEE7FEE7FEE727
S31508008320FEE7FEE7FEE7FEE7FEE7FEE7FEE7FEE717
S31508008330FEE7FEE7FEE7FEE7FEE7FEE7FEE7FEE707
S31508008340FEE7FEE7FEE7FEE7FEE7FEE7FEE7FEE7F7
S31508008350FEE7FEE7FEE7FEE7FEE7FEE7FEE7FEE7E7
S31508008360FEE700007C000020F0000020F0B50024A5
S3150800837021E0134D15F8147005EB440595F801E056
S3150800838007EB0E0505FB00054AF2104C9CFBF5F6BB
S3150800839005FB16C66EB99CFBF5F5ADB20D80013D21
S315080083A0ADB2B5F5806F04D2177083F800E00120EE
S315080083B0F0BD0134E4B2112CDBD90020F0BD00BFBA
S315080083C0388F0008F0B587B001214FF4003000F06F
S315080083D03FFC0121084600F02DFC1E4D0722022114
S315080083E0284600F023FA07220321284600F01EFA41
S315080083F000248DF8164001278DF8177002268DF88F
S315080084001460042304938DF8156004A9284600F027
S31508008410C7F98DF814600823049304A9284600F0C8
S31508008420BFF94FF461430093ADF80440ADF8064038
S31508008430ADF80840ADF80C400C23ADF80A30064CF0
S315080084406946204600F020FC3946204600F084FCA8
S3150800845007B0F0BD000002400044004070B58AB085
S315080084600121022000F0E6FB354E0922082130469C
S3150800847000F0DCF909221146304600F0D7F94FF42E
S315080084804073089302238DF824308DF82530002494
S315080084908DF8264001258DF8275008A9304600F0AA
S315080084A07FF929464FF0007000F0D2FBA6F5D036CA
S315080084B0304600F0D3F905A800F0EEFA6B460DEB4E
S315080084C005020DF102014FF4FA70FFF74FFF8DF820
S315080084D01A408DF81B408DF81C408DF81D408DF80C
S315080084E01E408DF81F408DF816408DF817409DF8F0
S315080084F00130013B8DF818309DF80030013B8DF8AE
S315080085001930BDF80230ADF8143005A9304600F030
S31508008510C1F98DF80E408DF80F408DF81050ADF862
S315080085200440ADF80640ADF80840ADF80A40ADF88D
S315080085300C408DF8115001A800F034FA0AB070BD4D
S315080085400004024010B504462021064800F016FC37
S31508008550012805D1034800F00DFC2070012010BD4C
S31508008560002010BD0044004008B5FFF72BFFFFF7B9
S3150800857075FF08BDBFF34F8F0449CA6802F4E0626D
S31508008580034B1343CB60BFF34F8FFEE700ED00E0CC
S315080085900400FA0508B5204B1B789BB91F48FFF75E
S315080085A0D1FF012836D11D4B1B78002B32D000F0A5
S315080085B0E7F81B4B18600122174B1A700022194B5B
S315080085C01A7008BD174B1B78013314481844FFF777
S315080085D0B9FF012814D1134A13780133DBB213709B
S315080085E00E4A1278934215D100220B4B1A700B4B88
S315080085F05B78FF2B0ED1094B9B785BB9FFF7BAFF67
S3150800860000F0BEF8064B1B686433984202D9002274
S31508008610014B1A7008BD00BFE1000020A000002031
S31508008620980000209C00002000B587B00021114862
S3150800863000F096FAD8B101AA00210E4800F03CFADB
S315080086409DF80C3033B940F26763019A9A4203D019
S31508008650002302E0002300E0012343B19DF80F3018
S31508008660FF2B04D19DF810300BB9FFF783FF07B035
S315080086705DF804FB0064004008B5FFF78BFFFFF7C1
S31508008680D3FF08BD08B500F00DF800F05BF808BD8B
S3150800869008B5FFF7F7FFFFF767FF00F025F8FFF7C4
S315080086A0EBFFFAE730B583B00121042000F0C2FAE7
S315080086B04FF48055009501238DF8043000228DF87B
S315080086C006208DF8073002238DF80530054C6946DB
S315080086D0204600F065F82946204600F0A3F803B0C6
S315080086E030BD00BF0008024010B500F049F80F4B36
S315080086F01B68C31AB3F5FA7F16D304460C4B1B78CE
S3150800870043B901220A4B1A704FF48051094800F008
S315080087108BF807E00022064B1A704FF48051054883
S3150800872000F080F8014B1C6010BD00BFE40000207B
S31508008730E800002000080240014B1860704700BF9F
S31508008740EC00002008B50A4B1B680A4AA2FB032363
S315080087509B09013B084A5360F021084B83F8231014
S315080087600020906007231360FFF7E6FF08BD00BFEF
S3150800877010000020D34D621010E000E000ED00E08C
S31508008780014B1868704700BFEC000020024A1368C6
S3150800879001331360704700BFEC000020FEE700BFFE
S315080087A070B400233AE001229A400C68A24334D1FF
S315080087B004685D000322AA40D24314400460066898
S315080087C00C79AC40344304600C79013CE4B2012CCA
S315080087D015D884682240826084684A79AA40224370
S315080087E0826046689AB20124944026EA04044460EA
S315080087F046688C7904FA02F292B232434260C4683F
S315080088009AB256000322B24024EA0202C260C6683F
S31508008810CC7904FA05F23243C26001330F2BC2D970
S3150800882070BC7047018370474183704730B401F0CC
S3150800883007039B009A40C908083150F821400F25C4
S3150800884005FA03F324EA030340F8213050F82130EF
S315080088501A4340F8212030BC704700BF08B50C4BBE
S3150800886098420AD101214FF0007000F0FFF900216B
S315080088704FF0007000F0FAF908BD01214FF0806052
S3150800888000F0F4F900214FF0806000F0EFF908BD20
S3150800889000640040036823F002030360036843F0A2
S315080088A001030360002300E00133426812F0010F60
S315080088B003D14FF6FF729342F6D1436813F0010FC6
S315080088C06BD08B79012B04D1036843F080030360D6
S315080088D003E0036823F080030360CB79012B04D1FE
S315080088E0036843F04003036003E0036823F0400392
S315080088F003600B7A012B04D1036843F0200303605D
S3150800890003E0036823F0200303604B7A012B04D1AC
S31508008910036843F01003036003E0036823F01003C1
S3150800892003608B7A012B04D1036843F008030360C4
S3150800893003E0036823F008030360CB7A012B04D114
S31508008940036843F00403036003E0036823F00403A9
S3150800895003608A78CB781B0643EA82730A7943EA6E
S3150800896002434A7943EA02530A88013A1343C36128
S31508008970036823F001030360002300E00133426823
S3150800898012F0010F03D04FF6FF729342F6D14368F7
S3150800899013F0010F03D00020704700207047012014
S315080089A0704700BF70B4837A012202FA03F3394A8A
S315080089B0D2F8001241F00101C2F80012D2F81C12D6
S315080089C0DC432140C2F81C12027BB2B9314AD2F804
S315080089D00C122140C2F80C12817AC688458845EAED
S315080089E00645483142F83150857A8688018841EA39
S315080089F00641483502EBC5025160027B012A16D1B1
S31508008A00244AD2F80C121943C2F80C12817A068845
S31508008A10458845EA0645483142F83150857A8688C0
S31508008A20C18841EA0641483502EBC5025160C27A5F
S31508008A3032B91849D1F804222240C1F8042205E0C7
S31508008A401449D1F804221A43C1F8042202892AB922
S31508008A501049D1F814221440C1F814420289012A97
S31508008A6005D10C49D1F814221A43C1F81422427BC5
S31508008A70012A05D10749D1F81C221343C1F81C3233
S31508008A80044AD2F8003223F00103C2F8003270BC5F
S31508008A90704700BF0064004000238371C3710372EE
S31508008AA043728372C3728370C370032303710223F4
S31508008AB0437101230380704710B401F11B031B01A6
S31508008AC0C35803F00403DBB2137233B901F11B0375
S31508008AD01B01C3585B0D136005E001F11B031B0165
S31508008AE0C358DB08536001F11B031B01C418C358A4
S31508008AF003F002035372636803F00F03937263680B
S31508008B001B0AD37400EB0113D3F8B841D472D3F817
S31508008B10B841240A1473D3F8B841240C5473D3F813
S31508008B20B841240E9473D3F8BC41D473D3F8BC412E
S31508008B30240A1474D3F8BC41240C5474D3F8BC31F9
S31508008B401B0E937421B9C36843F02003C36003E086
S31508008B50036943F0200303615DF8044B704700BFC7
S31508008B6019B9C06800F003007047012903D10069EC
S31508008B7000F0030070470020704700BF10B4294B6F
S31508008B809B6803F00C03042B05D0082B06D053BBB7
S31508008B90254B036029E0254B036026E0214B5A68E4
S31508008BA05B6803F03F0312F4800F09D01F4AB2FB3B
S31508008BB0F3F21C4B5B68C3F3881303FB02F208E06D
S31508008BC0194AB2FBF3F3174A5168C1F3881101FB3E
S31508008BD003F2144B5B68C3F3014301335B00B2FB3A
S31508008BE0F3F3036001E0104B03600E4CA368C3F374
S31508008BF003130F49CB5CDAB20368D3404360A2681B
S31508008C00C2F382228A5CD2B223FA02F28260A26896
S31508008C10C2F342328A5CD2B2D340C3605DF8044BD9
S31508008C20704700BF003802400024F40000127A00A2
S31508008C300000002021B1054B1A6B104318637047DA
S31508008C40024A136B23EA000010637047003802409B
S31508008C5021B1054B1A6C104318647047024A136C0D
S31508008C6023EA0000106470470038024021B1054B22
S31508008C701A6A104318627047024A136A23EA000008
S31508008C80106270470038024030B585B004460D467C
S31508008C90038A9BB223F44053CA8813430382838909
S31508008CA09BB223F4B05323F00C01A8882A896B8958
S31508008CB0024313430B43A381A38A9BB223F4407355
S31508008CC0AA891343A3826846FFF758FF204B9C42A4
S31508008CD003D003F580639C4201D1039A00E0029A0F
S31508008CE0A38913F4004F08D002EB820202EB82023A
S31508008CF029684900B2FBF1F107E002EB820202EBB8
S31508008D00820229688900B2FBF1F1124BA3FB012309
S31508008D105B091B011A09642000FB1212A18911F4D0
S31508008D20004F08D0D20032320A49A1FB0212C2F320
S31508008D3042121A4307E0120132320649A1FB021217
S31508008D40C2F343121A4392B2228105B030BD00BF66
S31508008D50001001401F85EB5129B183899BB243F46A
S31508008D6000538381704783899BB223F400539BB2D7
S31508008D70838170478088C0F30800704703881942CA
S31508008D8001D0012070470020704700BF82B0002341
S31508008D90019300932A4A136843F480331360284BDF
S31508008DA01B6803F400330093019B01330193009B76
S31508008DB01BB9019BB3F5A06FF1D1214B1B6813F4C6
S31508008DC0003F02D00123009301E000230093009B9B
S31508008DD0012B32D11A4B1A6C42F080521A64194987
S31508008DE00A6842F440420A609A689A609A6842F4AD
S31508008DF000429A609A6842F4A0529A60124A5A60EF
S31508008E001A6842F080721A600D4B1B6813F0007FD7
S31508008E10FAD040F205620D4B1A60A3F580639A6892
S31508008E2022F003029A609A6842F002029A60044BA2
S31508008E309B6803F00C03082BF9D102B0704700BFFA
S31508008E40003802400070004008544007003C0240C9
S31508008E5008B50F4AD2F8883043F47003C2F8883050
S31508008E600C4B1A6842F001021A60002199601A68D0
S31508008E7022F0847222F480321A60074A5A601A680D
S31508008E8022F480221A60D960FFF780FF08BD00BF70
S31508008E9000ED00E0003802401030002408B5074B0A
S31508008EA0044613B10021AFF30080054B1868836AA6
S31508008EB003B198472046FFF771FC00BF0000000089
S31508008EC05C8F000870B50E4B0E4CE41AA4100025F2
S31508008ED01E46A54204D056F8253098470135F8E7CE
S31508008EE000F01EF8084C094BE41AA41000251E468B
S31508008EF0A54204D056F8253098470135F8E770BDE5
S31508008F0074000020740000207800002074000020FF
S31508008F1002440346934202D003F8011BFAE770475E
S31508008F20F8B500BFF8BC08BC9E467047F8B500BF48
S31508008F30F8BC08BC9E4670470502060206030703EE
S31508008F400803090309040A040B040C040C050D059F
S31508008F500E050F050F06100610071008140000204E
S30908008F6000000000FF
S30D08008F6484F2FF7F0100000002
S31508008F6C00000000010203040102030406070809B5
S31508008F7C007A030A00000000000000000000000050
S31508008F8C00000000000000000000000000000000C7
S31508008F9C00000000000000000000000000000000B7
S31508008FAC00000000000000000000000000000000A7
S31508008FBC0000000000000000000000000000000097
S31508008FCC0000000000000000000000000000000087
S31108008FDC00000000B18100088D8100082B
S7050800800072
